:020000040800F2
:1000000000060020A1020008DD0F0008E10F000833
:1000100039100008E10F00080D100008A3020008C5
:10002000A3020008A3020008A3020008E5330008A9
:10003000A3020008A3020008A3020008A30200080C
:10004000A3020008A3020008A3020008A3020008FC
:10005000A3020008A3020008D537000801380008F1
:100060002D3800085938000885380008A302000818
:10007000A3020008A3020008A3020008A3020008CC
:10008000A3020008A3020008A3020008A3020008BC
:10009000A3020008A3020008A3020008B138000868
:1000A000A3020008A3020008A3020008A30200089C
:1000B000A3020008A3020008A3020008A30200088C
:1000C000A3020008A3020008A3020008A30200087C
:1000D000A3020008A3020008A3020008A30200086C
:1000E00019390008A3020008A3020008A3020008AF
:1000F000A3020008A3020008A3020008A30200084C
:10010000A3020008A302000861340008A30200084B
:10011000A3020008A3020008A3020008A30200082B
:10012000A3020008A3020008A3020008A30200081B
:10013000A3020008A3020008A3020008A30200080B
:10014000A3020008A3020008A3020008A3020008FB
:10015000A3020008A3020008A3020008A3020008EB
:10016000A3020008A3020008A3020008A3020008DB
:10017000A3020008592E0008A3020008A3020008E9
:10018000A3020008A3020008A3020008A3020008BB
:10019000A3020008A3020008A3020008A3020008AB
:1001A000A3020008A3020008A3020008A30200089B
:1001B000A3020008A3020008A3020008A30200088B
:1001C000A3020008A3020008A3020008A30200087B
:1001D000A3020008452E0008A3020008A30200089D
:1001E000A3020008A3020008A3020008A30200085B
:1001F000A3020008A3020008A3020008A30200084B
:10020000A3020008A3020008A3020008A30200083A
:10021000A3020008A3020008A3020008A30200082A
:10022000A3020008A3020008A3020008A30200081A
:10023000A3020008A3020008A3020008A30200080A
:10024000A3020008A3020008A3020008A3020008FA
:10025000A3020008A3020008A3020008A3020008EA
:10026000A3020008A3020008A3020008A3020008DA
:10027000A3020008A3020008A3020008A3020008CA
:10028000A3020008A3020008A3020008A3020008BA
:10029000A3020008A3020008A3020008A3020008AA
:1002A00002E000F000F8FEE772B6394880F30888F3
:1002B000384880F3098838484EF60851CEF20001DC
:1002C000086040F20000CCF200004EF63471CEF22D
:1002D00000010860BFF34F8FBFF36F8F40F2000043
:1002E000C0F2F0004EF68851CEF200010860BFF374
:1002F0004F8FBFF36F8F4FF00000E1EE100A4EF604
:100300003C71CEF200010860062080F31488BFF330
:100310006F8F02F043F802F0E3FF4FF055301F49B2
:100320001B4A91423CBF41F8040BFAE71C49194AA9
:1003300091423CBF41F8040BFAE71A491A4A1B4B99
:100340009A423EBF51F8040B42F8040BF8E7002034
:100350001749184A91423CBF41F8040BFAE702F0F2
:1003600061F803F031F8144C144DAC4203DA54F840
:10037000041B8847F9E700F03FF8114C114DAC42DF
:1003800003DA54F8041B8847F9E702F049B8000083
:1003900000060020002200200000000800000020CD
:1003A00000060020303D00080022002044220020EA
:1003B00048220020D82E0020A0020008A002000839
:1003C000A0020008A00200082DE9F04F2DED108AD0
:1003D000C1F80CD0D0F80CD0BDEC108ABDE8F08F7D
:1003E000002383F311882846A047002001F030FC49
:1003F00001F04CFB00DFFEE738B5204C6FF0010345
:10040000002523700323A57063701E23E5702571FA
:100410006571A571E57125726572A372E57200F0D0
:10042000D7FC20B10E2325726572A372E57201F02C
:1004300077FF044601F0ACFF0546D0B9104B9C4253
:1004400019D001339C4241F2883412BF0546002482
:100450000125002001F06EFF0DB100F05BF800F007
:100460008FFD00F0FDFB204600F014F900F052F87B
:10047000F9E70024EDE70446EBE700BF482200203F
:10048000010007B008B500F08DFBA0F12003584231
:10049000584108BD054B07B51B88022101A8ADF8DE
:1004A000043000F0CDFB03B05DF804FB1C3A0008FB
:1004B00010B5202383F311881248C3680BB101F0F3
:1004C0004DFC0023104A4FF47A710E4801F00AFCEB
:1004D000002383F311880D4C236813B12368013B7B
:1004E0002360636813B16368013B6360084B1B784A
:1004F00033B9636823B9022000F0AAFC3223636099
:1005000010BD00BF54220020B10400087023002059
:1005100068220020554B56492DE9F04153F8042F2D
:10052000013201D1BDE8F0818B42F7D1514C524BE1
:1005300022689A4240F29880504B9B6803F1006316
:1005400003F500339A4280F08F80002000F0A4FB76
:1005500002204B4B187000F06FFC4A4BD3F8E82098
:100560000022C3F8E820D3F81011C3F81021D3F803
:100570001011D3F8EC10C3F8EC20D3F81411C3F821
:100580001421D3F81411D3F8F010C3F8F020D3F8E5
:100590001811C3F81821D3F81811D3F8801041F0BE
:1005A0000061C3F88010D3F8801021F00061C3F817
:1005B0008010D3F88010D3F8801041F00071C3F898
:1005C0008010D3F8801021F00071C3F88010D3F8A8
:1005D000803072B62C4B2D490B601D682468BFF328
:1005E0004F8FBFF36F8F2A4BC3F88420BFF34F8F19
:1005F0005A6922F480325A61BFF34F8FD3F88020BA
:1006000043F6E07EC2F3C906C2F34E32B707520189
:1006100002EA0E0838463146013948EA000C00F17A
:100620004040B1F1FF3FC3F874C2F5D1203A12F156
:10063000200FEDD1BFF34F8FBFF36F8FBFF34F8FFD
:10064000BFF36F8F5A6922F400325A610022C3F857
:100650005022BFF34F8FBFF36F8F202383F3118896
:10066000AD4685F308882047BDE8F081FCFF01080E
:100670001C00020804000208FFFF010848220020B5
:1006800068220020004402580000020808ED00E043
:1006900000ED00E02DE9F04F99B0B34C2022FF218E
:1006A000019010A8A66800F00DFCB04AA34613788C
:1006B000A3B90121AE481170C360202383F31188D0
:1006C000C3680BB101F04AFB0023AA4A4FF47A71C8
:1006D000A74801F007FB002383F31188019B13B1A6
:1006E000A54B019A1A600023A44AA349019F994689
:1006F0001C461D46984613704B600292012000F084
:100700009BFB002F00F012829B4B1B68002B40F0DC
:100710000D8219B0BDE8F08F0220FFF7B3FE00286C
:1007200040F0FB81019BB9F1000F08BF1F46944BBD
:100730001B8802210BA8ADF82C3000F081FADDE710
:100740004FF47A7000F02EFA031E0393EADB0220C6
:10075000FFF798FE82460028E4D0039B581E042829
:1007600000F2DD81DFE800F0030E1114170018A875
:100770000523042140F8343D00F062FA54464FF05E
:10078000000856E004217848F6E704217D48F3E7A5
:1007900004217D48F0E71C242046043400F07EFA52
:1007A00004210B900BA800F04BFA2C2CF4D1E5E7B8
:1007B000002DB7D0002CB5D00220FFF763FE054610
:1007C000002800F0AF8101206C4C00F065FA4FF07A
:1007D00000090220207000F02FFB5FFA89FA5046D2
:1007E00000F06AFA074658B1504609F1010900F0D5
:1007F00073FA0028F1D12C46A9460027634B97E7EE
:1008000001233E460220237000F008FBDBF808308D
:100810009E4206D2304600F041FA0130EBD1043658
:10082000F4E70026029BA9462C461E703746524B21
:100830005E6000F09BFB15B1002C18BF0027FFF78E
:1008400029FE5BE7002D3FF46DAF002C3FF46AAF4B
:100850000220029B187000F0EFFA322000F0A2F99B
:10086000B0F1000AC0F25E811AF0030540F05A812F
:1008700006EB0A03DBF80820934200F25381BAF535
:10088000807F00F24F8155450DDA4FF47A7000F009
:1008900089F90490049B002BC0F24481049B3C4ADC
:1008A000AB540135EFE7C820FFF7ECFD0546002803
:1008B00000F038811F2E11D8C6F1200410AB26F0AD
:1008C000030033495445184428BF5446224600F0DB
:1008D000D1FA2246FF212E4800F0F4FA4FEAAA0A84
:1008E0002B4930465FFA8AF200F0F4FA04460028F9
:1008F00000F01A8106EB8A0605469AE70220FFF708
:10090000C1FD00283FF40EAF00F000FA00283FF4CC
:1009100009AF4FF0000A5346DBF8082092451CD27D
:10092000BAF11F0F12D8109A01320FD02AF0030229
:1009300018A90A4452F8202C0B92184604220BA93D
:100940000AF1040A00F08CFB0346E5E750460393E6
:1009500000F0A4F9039B0B90EFE718A8042140F8DE
:100960004C3D00F06DF964E7482200206C23002024
:1009700054220020B10400087023002068220020C7
:100980001E3A00084C22002050220020203A000885
:100990006C22002018A80023642140F8343D00F0A8
:1009A0002BF900287FF4BEAE0220FFF76BFD002874
:1009B0003FF4B8AE0B9800F0A1F918AB43F8480D1E
:1009C00004211846CDE718A80023642140F8343DDF
:1009D00000F012F900287FF4A5AE0220FFF752FDC7
:1009E00000283FF49FAE0B9800F08AF918AB43F84B
:1009F000440DE5E70220FFF745FD00283FF492AEE5
:100A000000F094F918AB43F8400DD9E70220FFF746
:100A100039FD00283FF486AE0BA9142000F08CF9B4
:100A2000824618A8042140F83CAD00F009F951466F
:100A30000BA896E7322000F0B5F8B0F1000AFFF6F7
:100A400071AE1AF0030F7FF46DAE0AEB0803DBF80A
:100A5000082093423FF666AE0220FFF713FD002800
:100A60003FF460AE2AF0030AC244D0453FF4E1AE41
:100A7000404608F1040800F011F904210A900AA880
:100A800000F0DEF8F1E74FF47A70FFF7FBFC002886
:100A90003FF448AE00F03AF900283FF4AFAE109BA7
:100AA00001330CD0082210A9002000F013FA00280E
:100AB0003FF4A4AE2022FF2110A800F003FAFFF7B4
:100AC000E9FC374801F0CAF823E6002D3FF42AAECE
:100AD000002C3FF427AE18A80023642140F8343DD1
:100AE00000F08AF8824600287FF41CAE0220FFF74F
:100AF000C9FC00283FF416AE0390FFF7CBFC41F28F
:100B00008830574601F0AAF80B9800F065FA00F01B
:100B10002DFA039B1C461D46F0E5054689E64FF07D
:100B20000008FFE52546FDE52C4667E6002000F0BD
:100B300039F80490049B002BFFF6E3AD012000F090
:100B40006DF9049B213B122B3FF6D8AD01A252F860
:100B500023F000BF1907000841070008B10700088B
:100B6000FD060008FD060008FD060008450800080F
:100B7000350A0008FD08000895090008C7090008A3
:100B8000F5090008FD0600080D0A0008FD0600082A
:100B9000870A000833080008FD060008CB0A000891
:100BA000A0860100114B37B51A78002401460132A6
:100BB0008DF80740D2B2012A11D80D4801220368EE
:100BC0001D6A4FF47A734B430DF10701A8470128C2
:100BD00005D1084B9DF807001C7003B030BD4FF4E1
:100BE000FA7001F03BF84FF0FF30F6E700220020EA
:100BF00060260020A423002038B50E4B05461A7845
:100C00000132D2B2012A0ED80B48042203681C6AB2
:100C10004FF47A734B432946A047042803D10020A0
:100C2000064B187038BD4FF4FA7001F017F84FF00A
:100C3000FF3038BD0022002060260020A4230020C1
:100C400030B4054C0A46014623682046DD69034B53
:100C5000AC4630BC604700BF60260020A086010083
:100C6000F8B50A4C00250A4E01F040FA094F2070F1
:100C700030682378834207D901F034FA3368054499
:100C80000133BD423360F3D9F8BD00BFA523002076
:100C900078230020FFFF010001F0F6BA00F10060A8
:100CA00000F500300068704700F10060920000F528
:100CB000003001F077BA0000054B1A68054B1B782D
:100CC0009B1A834202D9104401F00CBA00207047ED
:100CD00078230020A523002038B5074D0446286856
:100CE000204401F005FA28B928682044BDE83840BE
:100CF00001F010BA38BD00BF7823002000207047F3
:100D0000014BC058704700BF00E8F11F064991F839
:100D1000243033B100230822086A81F82430FFF719
:100D2000C3BF0120704700BF7C230020014B18681F
:100D3000704700BF0010005C234BF0B5234C1B68CC
:100D40002788C3F30B0665681B0C94F90820BE4284
:100D500028D0A789BE4206D101220C2505FB0244FA
:100D6000656894F9082041F20104A3421CD041F2C5
:100D70000304A3421AD042F20104A34218D042F263
:100D80000304A34208BF5622441E013D0B460C44F7
:100D9000A34217D215F9016F581C5EB1034600F843
:100DA000016CF5E70022D8E75A22EDE75922EBE77C
:100DB0005822E9E72C2584421D7001D9981C5A70ED
:100DC000401AF0BD1846FBE70010005C042200202A
:100DD000104B41F201015B888B429AB211D041F273
:100DE00003018B420FD042F201039A420DD042F22E
:100DF00003039A420BD10323074A02EB8303D878FB
:100E000070470023F8E70123F6E70223F4E7002008
:100E1000704700BF0010005C243A0008022804D18B
:100E20004FF48012034B9A6170470128FCD14FF4B4
:100E30000032F7E700040258022803D11022034BC6
:100E40009A6170470128FCD10222F8E70004025899
:100E5000022805D1064A536983F010035361704795
:100E60000128FCD1024A536983F00203F6E700BF70
:100E700000040258002310B5934203D0CC5CC45444
:100E80000133F9E710BD000030B5441E14F9010F1D
:100E90000B4658B193F900500131854206D11AB979
:100EA00093F90020801A30BD013AEFE7002AF7D10C
:100EB000104630BD02460346981A13F9011B00295B
:100EC000FAD1704702440346934202D003F8011B53
:100ED000FAE770472DE9F047234C05468846174648
:100EE00094F8243083BB2E46DFF87C90C7B394F887
:100EF00024302BB92022FF2148462662FFF7E2FF6B
:100F000094F824004146C0F1080504EB8000BD427E
:100F100028BF3D465FFA85FAAD00A7EB0A072A46CF
:100F20002E44FFF7A7FF94F82430A844FFB29A4458
:100F30005FFA8AFABAF1080F84F824A0D6D1FFF735
:100F4000E5FE0028D2D108E0266A06EB8306B0420F
:100F5000CAD0FFF7DBFE0028C5D10020BDE8F0872E
:100F60000120BDE8F08700BF7C230020024B1A78E7
:100F7000024B1A70704700BFA423002000220020FB
:100F800038B5114D114C284600F006F92146284687
:100F900000F02EF924680E48D4F89020D2F80438D6
:100FA00043F00203C2F8043800F058FE0949204615
:100FB00000F02EFAD4F89020D2F8043823F002037F
:100FC000C2F8043838BD00BF60260020F43A00089B
:100FD00040420F00143B000870470000FEE700008D
:100FE00000B59BB0EFF3098168226846FFF742FF26
:100FF000EFF30583044B9A6BDA6A9A6A9A6A9A6AE3
:101000009A6A9A6A9B6AFEE700ED00E000B59BB021
:10101000EFF3098168226846FFF72CFFEFF30583A1
:10102000044B9A6B9A6A9A6A9A6A9A6A9A6A9B6A53
:10103000FEE700BF00ED00E000B59BB0EFF30981D3
:1010400068226846FFF716FFEFF30583034B5A6BE0
:101050009A6A9A6A9A6A9A6A9B6AFEE700ED00E0C9
:1010600030B50A44074D91420BD011F8013B0924D9
:101070005840013CF7D040F300032B4083EA500076
:10108000F7E730BD2083B8ED002304491A465A50D3
:10109000C81808334260802BF9D17047A82300207C
:1010A000026843681143016003B1184770470000AC
:1010B00013B5446BD4F894341A681178042915D107
:1010C000217C022912D11979012312898B40134204
:1010D0000CD101A904F14C0002F006F8D4F89444B4
:1010E0000246019B2179206800F0EAF902B010BDA8
:1010F000143001F089BF00004FF0FF33143001F0CD
:1011000083BF00004C3002F05BB800004FF0FF33AB
:101110004C3002F055B80000143001F057BF000009
:101120004FF0FF31143001F051BF00004C3002F09D
:1011300027B800004FF0FF324C3002F021B8000019
:10114000D0F8942438B5136805461978042901D0DD
:10115000012038BD017C0229FAD1127901205C8975
:1011600090400440F4D105F1140001F0E9FE02467C
:101170000028EDD0D5F894544FF48073286869792D
:1011800000F08CF9204638BD406BFFF7D9BF000056
:1011900000207047704700007FB5124B01250226E2
:1011A000044603600023057400F18402436029466D
:1011B0008360C3600C4B0290143001934FF4807332
:1011C000009601F099FE094B04F52372294601931C
:1011D00004F14C004FF480730294009601F060FF1C
:1011E00004B070BD503A000889110008B110000821
:1011F0000A68202383F311880B790B3342F823000C
:101200004B79133342F823008B7913B10B3342F837
:1012100023000223C0F894140374002383F311887D
:101220007047000038B5037F044613B190F854307E
:10123000ABB90125201D0221FFF732FF04F1140094
:1012400025776FF0010100F031FD84F8545004F16E
:101250004C006FF00101BDE8384000F027BD38BDFB
:1012600010B5012104460430FFF71AFF002323774D
:1012700084F8543010BD000038B504460025143001
:1012800001F052FE04F14C00257701F021FF201DF2
:1012900084F854500121FFF703FF2046BDE8384091
:1012A000FFF74EBF90F8803003F06003202B19D178
:1012B00090F88120212A0AD0222A4FF000030ED074
:1012C000202A0FD1084A42670722826704E0064BB2
:1012D0004367072383670023C36701207047436781
:1012E0008367F9E7002070471C220020D0F894346F
:1012F00037B51A680446117804291AD1017C0229ED
:1013000017D11979012312898B40134211D100F1B1
:101310004C05284601F09CFF58B101A9284601F070
:10132000E3FED4F894440246019B2179206800F042
:10133000C7F803B030BD000001F10B03F7B550F85A
:10134000234005460E46F4B1202383F3118805EBB4
:101350008607201D08214C34FFF7A2FEFB685B695D
:101360001B6813B1204601F0CDFE01A9204601F013
:10137000BBFE024648B1019B3146284600F0A0F86A
:10138000002383F3118803B0F0BDFB685A6912682B
:10139000002AF5D01B8A013B1340F1D105F18002F0
:1013A000EAE70000133138B550F82140DCB12023C2
:1013B00083F31188D4F894241368527903EB8203E1
:1013C000DB689B695D6845B104216018FFF768FE22
:1013D000294604F1140001F0BDFD2046FFF7B0FEE0
:1013E000002383F3118838BD7047000001F0A2B8D4
:1013F000012300F1300200F150010370002343602B
:1014000042F8043B8A42D361FAD103814381704799
:1014100038B50446202383F31188002500F10C031E
:1014200000F13002416043F8045B9342FBD1204657
:1014300001F0A2F80223237085F3118838BD000063
:1014400070B500EB8103054650690E461446DA601C
:1014500018B110220021FFF735FDA06918B1102244
:101460000021FFF72FFD31462846BDE8704001F00E
:1014700095B90000038900F13002002103F0010357
:101480000381438903F00103438100F1100343F812
:10149000041B9342FBD101F019BA0000F0B40125FE
:1014A00000EB810447898D40E4683D43A469458190
:1014B00023600023A2606360F0BC01F035BA000035
:1014C000F0B4012500EB810407898D40E4683D43B9
:1014D0006469058123600023A2606360F0BC01F0B1
:1014E000ADBA0000022300F10C0200F1300110B58A
:1014F000037004460023A0F8883080F88A3080F812
:101500008B300381438142F8043B8A42FBD184F84B
:101510007030204601F0D6F863681B6823B120467E
:101520000021BDE81040184710BD00000278436854
:1015300080F88C2005221B6802700BB1042118472B
:1015400070470000436890F88C201B6802700BB154
:10155000052118477047000090F8703070B50446B8
:1015600013B1002380F8703004F18002204601F0AE
:10157000D1F963689B6863BB94F8805015F06006EE
:1015800015D194F8813005F07F0545EA032540F236
:1015900002339D4200F00E815BD8022D00F0DC800A
:1015A0003FD8002D00F08780012D00F0CF80002172
:1015B000204601F067FC0021204601F057FC6368DB
:1015C0001B6813B1062120469847062384F8703023
:1015D00070BD204698470028CED094F8872094F814
:1015E000863043EA0223A26F934238BFA36794F97F
:1015F0008030A56F002B4FF0200380F2FD80002D7E
:1016000000F0EC80092284F8702083F31188002117
:10161000A36F626F2046FFF753FF002383F3118807
:1016200070BDB5F5817F00F0B180B5F5407F49D040
:10163000B5F5807FBBD194F88230012BB7D1B4F8D7
:10164000883023F00203A4F888306667A667E6674F
:10165000C3E740F201639D421ED8B5F5C06F3BD28F
:10166000B5F5A06FA3D1B4F88030B3F5A06F0ED15B
:1016700094F88230204684F88A3001F081F863685B
:101680001B6813B1012120469847032323700023D0
:101690006367A367E367A0E7B5F5106F32D040F644
:1016A00002439D4252D0B5F5006F80D104F18B0307
:1016B0006367012324E004F18803E567636702237D
:1016C000A3678AE794F88230012B7FF470AFB4F8F7
:1016D000883043F00203B6E794F88520204661681D
:1016E00094F884304D6843EA022394F8831094F808
:1016F0008220A84700283FF45AAF43686367036815
:10170000A367A4E72378042B10D1202383F3118847
:101710002046FFF7AFFE86F311886368032184F843
:101720008B601B6821700BB12046984794F882307B
:10173000002BACD084F88B300423237063681B68C3
:10174000002BA4D0022120469847A0E7374B6367BF
:101750000223A36700239DE794F88410204611F02C
:10176000800F01F00F010ED001F0C6F8012806D05D
:1017700002287FF41CAF2E4BA067636767E72D4BF1
:10178000A567636763E701F0A9F8EFE794F8823093
:10179000002B7FF40CAF94F8843013F00F013FF46A
:1017A00076AF1A06204602D501F084FB6FE701F000
:1017B00075FB6CE794F88230002B7FF4F8AE94F858
:1017C000843013F00F013FF462AF1B06204602D5B0
:1017D00001F058FB5BE701F049FB58E7142284F85D
:1017E000702083F311882B462A4629462046FFF7AE
:1017F00055FE85F3118870BD5DB1152284F8702007
:1018000083F311880021A36F626F2046FFF746FE25
:1018100003E70B2284F8702083F311882B462A46B5
:1018200029462046FFF74CFEE3E700BF803A000858
:10183000783A00087C3A000838B590F870300446D1
:10184000152B29D8DFE803F03E28282828283E2831
:10185000280B293928282828282828283E3E90F8AF
:10186000871090F88620836F42EA01229A4214D9A9
:10187000C268128AB3FBF2F502FB15356DB920235D
:1018800083F311882B462A462946FFF719FE85F374
:1018900011880A2384F8703038BD142384F870301E
:1018A000202383F31188002320461A461946FFF7A8
:1018B000F5FD002383F3118838BDC36F03B198474A
:1018C0000023E7E7002101F0DDFA0021204601F0C6
:1018D000CDFA63681B6813B106212046984706239A
:1018E000D8E7000090F87020152A38B5044622D8B1
:1018F0000123934040F6416213421DD113F4801539
:101900000FD19B0217D50B2380F87030202383F36F
:1019100011882B462A462946FFF7D2FD85F3118808
:1019200038BDC3689B695B682BB9C36F03B1984727
:10193000002384F8703038BD002101F0A3FA0021A3
:10194000204601F093FA63681B6813B10621204614
:1019500098470623EDE70000024B00221B605B6006
:101960009A60704728240020002382680374054B86
:101970001B6899689142FBD25A680360426010600C
:10198000586070472824002008B5202383F311886D
:10199000037C032B05D0042B0DD02BB983F31188C6
:1019A00008BD436900221A604FF0FF334361FFF71F
:1019B000DBFF0023F2E790E80C001A600268536036
:1019C000F2E70000002382680374054B1B689968E6
:1019D0009142FBD85A6803604260106058607047BB
:1019E00028240020054B19690874186802685360A0
:1019F0001A60186101230374FEF7E6BC2824002056
:101A00004B1C30B5054687B00A4C10D0236901A89D
:101A1000094A00F067F92846FFF7E4FF049B13B179
:101A200001A800F09BF92369586907B030BDFFF7A2
:101A3000D9FFF8E7282400208919000838B50C4D93
:101A4000044641612B6981689A68914203D8BDE8D8
:101A50003840FFF789BF1846FFF786FF01232C6146
:101A6000014623742046BDE83840FEF7ADBC00BFF8
:101A700028240020044B1A681B6990689B689842D0
:101A800094BF0020012070472824002010B5084C86
:101A9000236820691A6854602260012223611A7445
:101AA000FFF790FF01462069BDE81040FEF78CBCAF
:101AB00028240020FEE7000010B5194CFFF74CFF6A
:101AC00000F002F980221749204600F087F8012330
:101AD00044F8180C0374144B144AD96821F4E061DB
:101AE0000904090C0A431249DA60CA6842F080729C
:101AF000CA60104A1049C2F8B01F116841F00101D4
:101B000011601022DA77202283F82220002383F349
:101B1000118862B60948BDE8104000F081B800BFE6
:101B200050240020843A000800ED00E00003FA058C
:101B3000F0ED00E0001000E055CEACC58C3A000896
:101B40002DE9F84F1E4C4FF00008DFF878906569DA
:101B500004F11407D9F82430266AAA689E1B96421D
:101B60001CD34FF0200AAA68236AD5F80CB0B61A25
:101B7000134423622B68BB425F606361C5F80C802D
:101B800001D101F091FB88F311882869D8478AF3C5
:101B900011886569AB689E42E5D2DBE76269BA42AB
:101BA0000CD0916823628E1B9660A86802282CBF17
:101BB0001818981CBDE8F84F01F07CBBBDE8F88F01
:101BC00028240020000C0040034B59685A68521A20
:101BD0009042FBD8704700BF001000E082600222F4
:101BE00002740022427470478368A3F17C0243F8B8
:101BF0000C2C026943F83C2C426943F8382C074A04
:101C000043F81C2CC268A3F1180043F8102C0222E0
:101C100003F8082C002203F8072C7047E1030008A2
:101C200010B5202383F31188FFF7DEFF002104465F
:101C3000FFF704FF002383F31188204610BD000046
:101C4000024B1B6958610F20FFF7CCBE28240020EF
:101C5000202383F31188FFF7F3BF000008B5014686
:101C6000202383F311880820FFF7CAFE002383F3A3
:101C7000118808BD49B1064B42681B6918605A605B
:101C8000136043600420FFF7BBBE4FF0FF30704786
:101C9000282400200368984206D01A680260506029
:101CA00018465961FFF760BE7047000038B504461A
:101CB0000D462068844200D138BD036823605C6013
:101CC0004561FFF751FEF4E7054B03F114025A6139
:101CD0009A614FF0FF32DA6100221A62704700BF4A
:101CE00028240020F8B5036102291A4B0646C26079
:101CF00038BF02215C6A184B1A461F4652F8145F1F
:101D000095420AD1586198611C6205604560816006
:101D10000819BDE8F84001F0BDBA186AAB68241A8A
:101D20000C1902D3E41A2D6804E09C4202D220442C
:101D300001F0C0FAAB689C42F4D86B683560736000
:101D40001E604FF0FF336E60B460A968091BA96084
:101D5000FB61F8BD000C00402824002010B41A4C90
:101D6000234653F8141F814210D0416802680A606C
:101D7000026851609A424FF00001C16003D093683D
:101D800081680B4493605DF8044B70470A6800203B
:101D90009A4262615360C86003D15DF8044B01F060
:101DA00083BA936888680344206A9360074A526A3A
:101DB000121A9342E7D9991A5DF8044B012998BF8A
:101DC000931C184401F076BA28240020000C00402F
:101DD00000207047FEE70000704700004FF0FF3022
:101DE00070470000022906D0032906D001290648C1
:101DF00018BF0020704705487047032A9ABF04485F
:101E000000EBC20000207047703B0008243B000834
:101E10002422002070B59AB006460846144601AD4B
:101E2000294600F095F82846FFF744F8C0B2431C55
:101E30005B0086E8180023700323023404F8013C99
:101E400000231946DAB20234904201D81AB070BDAC
:101E5000EA5C013304F8011C04F8022CF2E70000EC
:101E600008B5202383F311880348FFF73FFA0023C6
:101E700083F3118808BD00BF6026002010B504461A
:101E8000052916D8DFE801F016150316161D2023C4
:101E900083F311880E4A0121FFF7D2FA20460D4A3A
:101EA0000221FFF7CDFA0C48FFF7E6F9002383F390
:101EB000118810BD202383F311880748FFF7B2F97A
:101EC000F4E7202383F311880348FFF7C9F9EDE70E
:101ED000AC3A0008D03A00086026002038B50C4D16
:101EE0000C4C2A460C4904F10800FFF793FF05F15A
:101EF000CA0204F110000949FFF78CFF05F5CA7208
:101F000004F118000649BDE83840FFF783BF00BF61
:101F1000282B002024220020FC3A0008003B000867
:101F20000B3B000870B5044608460D46FEF7C2FF9D
:101F3000C6B22046013403780BB9184670BD32464C
:101F40002946FEF7A1FF0028F3D1012070BD000053
:101F50002DE9F04704460D46FEF7ACFF2B49C6B20B
:101F60002046FFF7DFFF08B10E36F6B228492046BB
:101F7000FFF7D8FF08B11036F6B2632E0BD8DFF8A2
:101F80008C80DFF88C90234FDFF894A0267846B938
:101F90002E70BDE8F08721462846BDE8F04701F0E5
:101FA00035BD252E2ED1072241462046FEF76CFF77
:101FB00070B9194B2A4603F1140153F8040B8B42F4
:101FC00042F8040BF9D11B78073415351370DDE79F
:101FD000082249462046FEF757FF98B9AA1C0F4B26
:101FE00013F8011F023209095345C95D02F8041CA8
:101FF000197801F00F01C95D02F8031CF0D1183502
:102000000834C3E72E7001340135BFE7903B000868
:102010000B3B0008AE3B0008983B0008FFE7F11FB0
:102020000BE8F11FBFF34F8F044B1A695107FCD126
:10203000D3F810215207F8D1704700BF002000529A
:1020400008B50D4B1B78ABB9FFF7ECFF0B4BDA680B
:10205000D10704D50A4A5A6002F188325A60D3F88F
:102060000C21D20706D5064AC3F8042102F18832B2
:10207000C3F8042108BD00BF862D002000200052B7
:102080002301674508B5114B1B78F3B9104B1A694A
:10209000510703D5DA6842F04002DA60D3F8102124
:1020A000520705D5D3F80C2142F04002C3F80C21A9
:1020B000FFF7B8FF064BDA6842F00102DA60D3F8A6
:1020C0000C2142F00102C3F80C2108BD862D00202E
:1020D000002000520F289ABF00F5806040040020C5
:1020E000704700004FF40030704700001020704728
:1020F0000F2808B50BD8FFF7EDFF00F50033026895
:10210000013204D104308342F9D1012008BD0020FE
:1021100008BD00000F2810B504463FD8FFF782FF26
:10212000FFF78EFF1E484FF0FF33072C4361C0F8C6
:1021300014311DD80361FFF775FF230243F0240318
:10214000C360C36843F08003C36003695A07FCD4CB
:10215000FFF768FF2046FFF7BDFF4FF4003100F0A6
:10216000F9F8FFF78FFF2046BDE81040FFF7C0BF2A
:10217000C0F81031FFF756FFA4F108031B0243F02B
:102180002403C0F80C31D0F80C3143F08003C0F8C0
:102190000C31D0F810315B07FBD4D9E7002010BD1B
:1021A000002000522DE9F84F40EA02030546894617
:1021B0009046DB065AD122F00302034602449342C2
:1021C00005D1FFF73DFF4E46DFF8B8B042E0196891
:1021D00001314BD10433F2E7264A05F17843264812
:1021E0009342264B264F88BF9A46A3F1FC039CBF1F
:1021F000DA46184603F1F80388BF1F46FFF712FFBF
:102200004FF0FF3306F11C02A5EB060E03603B689E
:1022100043F002033B60331FDAF8004014F005047A
:10222000FAD153F8041F9A424EF80310F4D1BFF3C9
:102230004F8FFFF7F7FE4FF0FF3320223146036048
:1022400028463B6823F002033B6001F0CFFB58B9FE
:1022500020352036A8EB06034B441F2BBCD80120A9
:10226000FFF710FFBDE8F88F2046F9E70020BDE832
:10227000F88F00BFFFFF0F00142100521021005201
:102280000C2000521020005210B5084C237828B1C1
:1022900053B9FFF7D5FE0123237010BD23B1207081
:1022A000BDE81040FFF7EEBE10BD00BF862D002038
:1022B00002440439064BD2B210B5904200D110BD91
:1022C000441C00B253F8200041F8040FE0B2F4E7D8
:1022D000504000580F4B30B51C6F240405D41C6FC0
:1022E0001C671C6F44F400441C670B4C0244043907
:1022F0002368D2B243F480732360084B904200D12C
:1023000030BD441C51F8045F00B243F82050E0B2E5
:10231000F4E700BF004402580048025850400058FB
:1023200007B5012201A90020FFF7C2FF019803B001
:102330005DF804FB13B50446FFF7F2FFA04206D098
:1023400002A90122002041F8044DFFF7C3FF02B0AB
:1023500010BD00000144BFF34F8F064B884204D3E9
:10236000BFF34F8FBFF36F8F7047C3F85C0220300D
:10237000F4E700BF00ED00E0034B1B685B0142BFC8
:102380000122024B1A707047D0440258872D00205A
:10239000014B1878704700BF872D0020F0B5BFF3C0
:1023A0004F8FBFF36F8F1D4B0021C3F85012BFF347
:1023B0004F8FBFF36F8F5A6942F400325A61BFF3F7
:1023C0004F8FBFF36F8FC3F88410BFF34F8FD3F8D5
:1023D000802043F6E076C2F3C904C2F34E32A5076B
:1023E000520102EA060E284621464EEA000701394C
:1023F00000F14040C3F860724F1CF6D1203A12F150
:10240000200FEED1BFF34F8F5A6942F480325A61E8
:10241000BFF34F8FBFF36F8FF0BD00BF00ED00E043
:10242000FEE70000084A094B09498B4204D3094AD8
:102430000021934205D3704752F8040F43F8040B70
:10244000F3E743F8041BF4E7703D0008D82E0020A2
:10245000D82E0020D82E0020D0F89430002230B59D
:102460001146D0F890409D684FF0FF3004EB4213C6
:1024700001329542C3F80019C3F81019C3F80809CE
:10248000C3F8001BC3F8101BC3F8080BEED24FF0C3
:102490000113C4F81C3830BD00EB81032DE9F04F67
:1024A000D3F80CE04F1C4FEA4118DEF814403F030C
:1024B000D4F800C06568D0F8902065450AD30120A3
:1024C000D2F8343800FA01F123EA0101C2F83418D5
:1024D000BDE8F08FACEB0503BEF81060B34228BF37
:1024E000334602EB0806D6F81869B6B2B3EB860F8E
:1024F00013D8A6683A449946A6F1040A5AF804BFCC
:10250000B9F1040FC2F800B002D9A9F10409F5E746
:102510001E442B44A6606360CCE70020BDE8F08F2A
:10252000890141F02001016103699B06FCD412205E
:10253000FFF74ABB10B50A4C2046FEF759FF094B7E
:10254000C4F89030084BC4F89430084C2046FEF78D
:102550004FFF074BC4F89030064BC4F8943010BDC1
:10256000882D002000000840E43B0008242E0020B5
:1025700000000440F03B00080378012B70B50546CD
:102580005DD1494BD0F89040984259D1474B0E212C
:102590006520D3F8D82042F00062C3F8D820D3F8E1
:1025A000002142F00062C3F80021D3F80021D3F8E3
:1025B000802042F00062C3F88020D3F8802022F00F
:1025C0000062C3F88020D3F8803000F07FFC384BE5
:1025D000E360384BC4F800380023D5F89060C4F8A5
:1025E000003EC02323604FF40413A3633369002B20
:1025F000FCDA01230C203361FFF7E6FA3369DB07CD
:10260000FCD41220FFF7E0FA3369002BFCDA002635
:102610002846A660FFF720FF6B68C4F81068DB68E7
:10262000C4F81468C4F81C68002B3AD1224BA3618B
:102630004FF0FF336361A36843F00103A36070BDF3
:102640001E4B9842C8D1194B0E214D20D3F8D820EB
:1026500042F00072C3F8D820D3F8002142F0007293
:10266000C3F80021D3F80021D3F8802042F0007293
:10267000C3F88020D3F8802022F00072C3F88020B5
:10268000D3F88020D3F8D82022F08062C3F8D82075
:10269000D3F8002122F08062C3F80021D3F8003182
:1026A00093E7074BC3E700BF882D00200044025882
:1026B0004014004003002002003C30C0242E0020C3
:1026C000083C30C0F8B5D0F89040054600214FF0E6
:1026D00000662046FFF724FFD5F8941000234FF042
:1026E00001128F684FF0FF30C4F83438C4F81C284A
:1026F00004EB431201339F42C2F80069C2F8006B39
:10270000C2F80809C2F8080BF2D20B68D5F890207D
:10271000C5F89830636210231361166916F010062D
:10272000FBD11220FFF750FAD4F8003823F4FE63EF
:10273000C4F80038A36943F4402343F01003A361B5
:102740000923C4F81038C4F814380B4BEB604FF071
:10275000C043C4F8103B094BC4F8003BC4F81069EF
:10276000C4F80039D5F8983003F1100243F480130F
:10277000C5F89820A362F8BDC03B00084080001057
:10278000D0F8902090F88A10D2F8003823F4FE6335
:1027900043EA0113C2F80038704700002DE9F04108
:1027A0000EB20D4600EB8608D8F80C100F6807F043
:1027B0000303022B53D0032B53D03F4A3F4F012B2F
:1027C00018BF1746D0F890404FEA451E002205F189
:1027D000100C04EB0E03C3F8102B8A69002A42D0B8
:1027E0004A8A05F158033A435B01E2500123D4F8C9
:1027F0001C2803FA0CF31343C4F81C38A644002326
:102800004A69CEF8103905F13F03002A3BD00A8A05
:1028100004EB8303898B9208012988BF4A43D0F8CF
:102820009810561841EA02422946C0F8986020469E
:102830005A60FFF775FED8F80C301B8A43EA8553BF
:102840001F4305F148035B01E7500123D4F81C281E
:1028500003FA05F51543C4F81C58BDE8F081184F7C
:10286000B0E7184FAEE704EB4613D3F8002B22F481
:102870000042C3F8002B0123D4F81C2803FA0CF300
:1028800022EA0303B8E704EB83030F4A04EB46167E
:1028900029465A602046FFF743FED6F80039012248
:1028A00023F4004302FA05F5C6F80039D4F81C38C1
:1028B00023EA0505CFE700BF008000100080041068
:1028C0000080081000800C1000040002D0F8942052
:1028D0001268C0F89820FFF7BFBD00005831D0F84B
:1028E000903049015B5813F4004004D013F4001FEA
:1028F00014BF0120022070474831D0F890304901C0
:102900005B5813F4004004D013F4001F14BF0120DF
:102910000220704700EB8101CB68196A0B681360D5
:102920004B6853607047000000EB810330B5DD68F1
:10293000AA691368D36019B9402B84BF4023136080
:102940006B8A1468D0F890201C4402EB4110013CC3
:1029500009B2B4FBF3F46343033323F0030343EA04
:10296000C44343F0C043C0F8103B2B6803F003039B
:10297000012B0ED1D2F8083802EB411013F4807FFE
:10298000D0F8003B14BF43F0805343F00053C0F82D
:10299000003B02EB4112D2F8003B43F00443C2F883
:1029A000003B30BD2DE9F041D0F8906005460C4663
:1029B00006EB4113D3F8087B3A07C3F8087B08D528
:1029C000D6F814381B0704D500EB8103DB685B687D
:1029D0009847FA072FD5D6F81438DB072BD505EB27
:1029E0008403D968CCB98B69488A5E68B6FBF0F27B
:1029F00000FB12628AB91868DA6890420DD2121A86
:102A000083E81400202383F3118821462846FFF72A
:102A10008BFF84F31188BDE8F081012303FA04F2EF
:102A20006B8923EA02036B81CB6823B121462846D8
:102A3000BDE8F0411847BDE8F081000000EB8103DC
:102A40004A0170B5DD68D0F890306C692668E660A0
:102A500056BB1A444FF40020C2F810092A6802F04D
:102A60000302012A0AB20ED1D3F8080803EB42147C
:102A700010F4807FD4F8000914BF40F0805040F07B
:102A80000050C4F8000903EB4212D2F8000940F0EC
:102A90000440C2F800090122D3F8340802FA01F117
:102AA0000143C3F8341870BD19B9402E84BF4020CB
:102AB000206020681A442E8A841940F00050013C9E
:102AC000B4FBF6F440EAC440C6E700002DE9F0414B
:102AD000D0F8906004460D4606EB4113D3F8087910
:102AE000C3F80879FB071CD5D6F81038DA0718D5D3
:102AF00000EB8103D3F80CE0DEF81430D3F800C00B
:102B0000DA6894451BD2A2EB0C024FF000081A6061
:102B1000C3F80480202383F31188FFF78FFF88F325
:102B200011883B0618D50123D6F83428AB40134250
:102B300012D029462046BDE8F041FFF7ADBC012385
:102B400003FA01F2038923EA02030381DEF8083065
:102B5000002BE6D09847E4E7BDE8F0812DE9F04787
:102B6000D0F8905004466E69AB691E40F1046E6166
:102B700003D5BDE8F047FEF7B5BC002E12DAD5F854
:102B8000003E9A0705D0D5F8003E23F00303C5F8B0
:102B9000003ED5F80438204623F00103C5F8043878
:102BA000FEF7D0FC330502D52046FEF7BFFCB70484
:102BB0000CD5D5F8083813F0060FEB6823F47053E2
:102BC0000CBF43F4105343F4A053EB60300704D51B
:102BD0006368DB680BB120469847F10200F1A180E1
:102BE000B2020BD5D4F8908000274FF00109D4F839
:102BF0009430F9B29B688B4280F0D280F3061AD5EC
:102C0000D4F890100A6AC2F30A1702F00F0302F414
:102C1000F012B2F5802F00F0EB80B2F5402F0AD110
:102C200004EB830301F58051DB68186A00231A4620
:102C30009F4240F0D1803003D5F8185835D5E903CC
:102C400003D500212046FFF7ADFEAA0303D50121DD
:102C50002046FFF7A7FE6B0303D502212046FFF7AE
:102C6000A1FE2F0303D503212046FFF79BFEE802B8
:102C700003D504212046FFF795FEA90203D50521BF
:102C80002046FFF78FFE6A0203D506212046FFF794
:102C900089FE2B0203D507212046FFF783FEEF01B3
:102CA00003D508212046FFF77DFE700340F1C78061
:102CB000E90703D500212046FFF708FFAA0703D53F
:102CC00001212046FFF702FF6B0703D502212046B2
:102CD000FFF7FCFE2F0703D503212046FFF7F6FE82
:102CE000EE0603D504212046FFF7F0FEA80603D523
:102CF00005212046FFF7EAFE690603D50621204696
:102D0000FFF7E4FE2A0603D507212046FFF7DEFE83
:102D1000EB0540F1948020460821BDE8F047FFF71D
:102D2000D5BED4F890904FF000084FF0010AD4F8C7
:102D300094305FFA88F79B68BB42FFF451AF09EB10
:102D40004713D3F8002902F44022B2F5802F24D192
:102D5000D3F80029002A20DAD3F8002942F0904263
:102D6000C3F80029D3F80029002AFBDB3946D4F840
:102D70009000FFF7D5FB22890AFA07F322EA030342
:102D8000238104EB8703DB689B6813B13946204637
:102D9000984739462046FFF77FFB08F10108C6E750
:102DA00008EB4112D2F8003B03F44023B3F5802F27
:102DB00010D1D2F8003B002B0CDA628909FA01F33A
:102DC00022EA0303638104EB8103DB68DB680BB158
:102DD0002046984701370AE713F0030F00D10A682D
:102DE000072B03F101039EBF0270120A01301FE797
:102DF00004EB830301F58051DA6890690268D0F82A
:102E000008C04068A2EB000E00221046974208D18D
:102E1000DB689B699A683A449A605A6817445F6015
:102E200009E712F0030F00D10868964502F101028C
:102E300082BF8CF80000000A0CF1010CE6E7BDE847
:102E4000F087000008B50348FFF788FEBDE808409A
:102E500000F0D8BA882D002008B50348FFF77EFEA1
:102E6000BDE8084000F0CEBA242E0020D0F8903003
:102E700003EB4111D1F8003B43F40013C1F8003BD0
:102E800070470000D0F8903003EB4111D1F80039C1
:102E900043F40013C1F8003970470000D0F89030B7
:102EA00003EB4111D1F8003B23F40013C1F8003BC0
:102EB00070470000D0F8903003EB4111D1F8003991
:102EC00023F40013C1F800397047000000F160439B
:102ED00000F01F020901400903F56143C9B28000F7
:102EE00083F80013012300F16040934000F5614036
:102EF000C0F880310360704730B50433039C017221
:102F0000002104FB0325C361049B00600363059B50
:102F10004060C16042610261856104624262816217
:102F2000C162436330BD00000022416AC26041615A
:102F300001616FF001018262C262FEF7B7BE00005C
:102F400003694269934203D1C2680AB10020704705
:102F5000181D7047036919600021C2680132C26000
:102F6000C269134482699342036124BF436A0361C7
:102F7000FEF790BE38B504460D46E3683BB1626982
:102F80000020131D1268A3621344E36238BD237A44
:102F900033B929462046FEF76DFE0028EDDA38BD2C
:102FA0006FF00100FBE70000C368C269013BC3602A
:102FB0004369134482699342436124BF436A436176
:102FC00000238362036B03B11847704770B5202359
:102FD000044683F31188866A3EB9FFF7CBFF0546A6
:102FE00018B186F31188284670BDA36AE26A13F807
:102FF000015B9342A36202D32046FFF7D5FF002373
:1030000083F31188EFE700002DE9F84F04460E46E0
:1030100090469946202787F311880025AA46D4F8C0
:1030200028B0BBF1000F09D149462046FFF7A2FFA7
:1030300020B18BF311882846BDE8F88FA16AA8EB70
:10304000050BE36A5B1A9B4528BF9B46BBF1400F0B
:103050001BD9334601F1400251F8040B914243F869
:10306000040BF9D1A36A403640354033A362A26A0B
:10307000E36A9A4202D32046FFF796FF8AF311884B
:103080004545D8D287F31188C9E730465A46FDF73F
:10309000F1FEA36A5E445D445B44A362E7E700007F
:1030A00010B5029C04330172C36103FB04210023A9
:1030B00000608362C362039B40600363049BC4603F
:1030C00042610261816104624262436310BD00009B
:1030D000026A6FF00101C260426A4261026100222D
:1030E0008262C262FEF7E2BD436902699A4203D17D
:1030F000C2680AB100207047184650F8043B0B60C4
:1031000070470000C3680021C2690133C36043698E
:10311000134482699342436124BF436A4361FEF7CB
:10312000B9BD000038B504460D46E3683BB12369DC
:1031300000201A1DA262E2691344E36238BD237ABB
:1031400033B929462046FEF795FD0028EDDA38BD53
:103150006FF00100FBE7000003691960C268013AE3
:10316000C260C269134482699342036124BF436A07
:10317000036100238362036B03B1184770470000AB
:1031800070B5202304460E4683F31188856A35B94D
:103190001146FFF7C7FF10B185F3118870BDA36A10
:1031A0001E70A36AE26A01339342A36204D3E16909
:1031B00020460439FFF7D0FF002080F3118870BD4E
:1031C0002DE9F84F04460D4691469A464FF02008E7
:1031D00088F311880026B346A76A4FB951462046A6
:1031E000FFF7A0FF20B187F311883046BDE8F88FC4
:1031F000A06AA9EB0603E76A3F1A9F4228BF1F4651
:10320000402F1BD905F1400355F8042B9D4240F88F
:10321000042BF9D1A36A40364033A362A26AE36A61
:103220009A4204D3E16920460439FFF795FF8BF3F6
:1032300011884E45D9D288F31188CDE729463A4600
:10324000FDF718FEA36A3D443E443B44A362E5E714
:10325000026943699A4203D1C3681BB91846704793
:103260000023FBE7836A002BF8D0043B9B1AF5D0C0
:103270001360C368013BC360C3691A4483699A42FF
:10328000026124BF436A0361002383620123E5E7EF
:1032900000F0FAB8034B002258631A610222DA6088
:1032A000704700BF000C00400022014BDA607047FD
:1032B000000C0040014B5863704700BF000C0040F9
:1032C0004B6843608B688360CB68C3600B69436164
:1032D0004B6903628B6943620B68036070470000AF
:1032E00008B52C4B40F2FF712B48D3F888200A43D5
:1032F000C3F88820D3F8882022F4FF6222F0070266
:10330000C3F88820D3F88820D3F8E0200A43C3F814
:10331000E020D3F808210A43C3F808211F4AD3F854
:1033200008311146FFF7CCFF1D4802F11C01FFF7E1
:10333000C7FF1C4802F13801FFF7C2FF1A4802F12B
:103340005401FFF7BDFF194802F17001FFF7B8FF04
:10335000174802F18C01FFF7B3FF164802F1A801EC
:10336000FFF7AEFF144802F1C401FFF7A9FF1348AD
:1033700002F1E001FFF7A4FF114802F1FC01FFF7A1
:103380009FFF104802F58C71FFF79AFFBDE80840D7
:1033900000F054B90044025800000258FC3B0008F9
:1033A0000004025800080258000C0258001002588D
:1033B0000014025800180258001C0258002002583D
:1033C000002402580028025808B500F0FFFAFEF762
:1033D00073FBFEF7D1FFBDE80840FEF77FBD00009C
:1033E00070470000064A536823F001035360EFF36F
:1033F0000983683383F30988002383F311887047B6
:1034000030EF00E010B5202383F31188104B5B6888
:1034100013F4006318D0F1EE103AEFF309844FF083
:10342000807344F84C3C0B4BDB6844F8083CA4F137
:10343000680383F30988FEF71DFB18B1064B44F8B7
:10344000503C10BD054BFAE783F3118810BD00BF57
:1034500000ED00E030EF00E0F1030008F4030008A5
:10346000084B1A69920710B508D500241C61202367
:1034700083F31188FEF764FB84F31188BDE81040E4
:10348000FFF7C0BF000C0040124B08213220D3F8D8
:10349000E82042F00802C3F8E820D3F8102142F0F7
:1034A0000802C3F810210C4AD3F81031D36B43F053
:1034B0000803D363C722094B9A624FF0FF32DA62E6
:1034C00000229A615A63DA605A6001225A611A60D6
:1034D000FFF7FCBC004402580010005C000C0040E8
:1034E000F8B5514B0024D3F880204FF0FF32C3F8D9
:1034F0008020D3F88010C3F88040D3F88010D3F830
:103500008410C3F88420D3F88410C3F88440D3F81F
:103510008410D96F41F0FF4141F4FF0141F4DF41D4
:1035200041F07F01D967D96F21F0FF4121F4FF01FC
:1035300021F4DF4121F07F01D967D96FD3F88810DA
:103540006FEA41516FEA5151C3F88810D3F88810DF
:10355000C1F30A01C3F88810D3F88810D3F890108B
:10356000C3F89020D3F89010C3F89040D3F890108F
:10357000D3F89410C3F89420D3F89410C3F894406F
:10358000D3F89410D3F89810C3F89820D3F8981073
:10359000C3F89840D3F89810D3F88C10C3F88C2057
:1035A000D3F88C10C3F88C40D3F88C10D3F89C104F
:1035B000C3F89C20D3F89C20C3F89C40D3F89C30DF
:1035C00000F0E4F9194B07229A60194ADA60194AA7
:1035D0001A6105225A60184A536A43F480335362D1
:1035E000C2F88440BFF34F8FD2F8803043F6E076C4
:1035F000C3F3C904C3F34E33A5075B0103EA060E08
:10360000284621464EEA0007013900F14040C2F841
:1036100074724F1CF6D1203B13F1200FEED1BFF393
:103620004F8FBFF36F8FF8BD0044025890ED00E05C
:10363000000004301D00080300ED00E00122574B9C
:1036400057491A60574B19609A60574ADA6000224E
:103650001A614FF440429A619A699004FCD51A6845
:1036600042F480721A60514B1A6F12F4407F04D0FA
:103670004FF480321A6700221A671A6842F001027A
:103680001A604A4A134611684907FCD500211161A6
:103690001A6912F03802FBD1012119604FF0804104
:1036A00059605A67424ADA62424A1A611A6842F419
:1036B00080321A603D4B1A689203FCD53E4A3F495E
:1036C0009A6200225A631963A1F58021DA634B39AB
:1036D00099635A643A4A1A643A4ADA621A6842F0BA
:1036E000A8521A60314B1A6802F02852B2F1285FD2
:1036F000F9D1482222219A614FF48862DA6140228E
:103700001A624FF00052DA641A652F4A5A652F4A3E
:103710009A652F4A11601A6942F003021A61234B1D
:103720001A6902F03802182AFAD1D3F8DC2042F0E4
:103730000052C3F8DC20D3F8042142F00052C3F851
:103740000421D3F80421D3F8DC2042F08042C3F8EE
:10375000DC20D3F8042142F08042C3F80421D3F8DE
:103760000421D3F8DC2042F00042C3F8DC20D3F877
:10377000042142F00042C3F80421D3F80421D3F815
:10378000F42042F00202C3F8F420D3F81C2142F0E6
:103790000202C3F81C21D3F81C3170470881005184
:1037A00000C000F000480258020000010044025826
:1037B0000000FF01008890083230600063020701BA
:1037C00047040508FD0BFF010010E00000010100A7
:1037D00000200052084A08B5936811680B4003F0B6
:1037E0000103936023B1054A13680BB150689847F1
:1037F000BDE80840FFF706BE80000058A82300205F
:10380000084A08B5936811680B4003F002039360FF
:1038100023B1054A93680BB1D0689847BDE80840CA
:10382000FFF7F0BD80000058A8230020084A08B523
:10383000936811680B4003F00403936023B1054AB9
:1038400013690BB150699847BDE80840FFF7DABD2E
:1038500080000058A8230020084A08B59368116822
:103860000B4003F00803936023B1054A93690BB141
:10387000D0699847BDE80840FFF7C4BD80000058F4
:10388000A8230020084A08B5936811680B4003F08C
:103890001003936023B1054A136A0BB1506A98472D
:1038A000BDE80840FFF7AEBD80000058A823002007
:1038B000174B10B59C681A68144004F478729A602B
:1038C000A30604D5134A936A0BB1D06A98476006E1
:1038D00004D5104A136B0BB1506B9847210604D5E1
:1038E0000C4A936B0BB1D06B9847E20504D5094A9B
:1038F000136C0BB1506C9847A30504D5054A936C23
:103900000BB1D06C9847BDE81040FFF77BBD00BFFE
:1039100080000058A82300201A4B10B59C681A6834
:10392000144004F47C429A60620504D5164A136D73
:103930000BB1506D9847230504D5134A936D0BB115
:10394000D06D9847E00404D50F4A136E0BB1506E4A
:103950009847A10404D50C4A936E0BB1D06E9847DA
:10396000620404D5084A136F0BB1506F98472304C3
:1039700004D5054A936F0BB1D06F9847BDE810404E
:10398000FFF740BD80000058A8230020062108B59D
:103990000846FFF79BFA06210720FFF797FA062152
:1039A0000820FFF793FA06210920FFF78FFA062176
:1039B0000A20FFF78BFA06211720FFF787FA062166
:1039C0002820BDE80840FFF781BA000008B5FFF7DE
:1039D00087FDFDF759FBFDF709FDFDF7DBFBFFF761
:1039E000FFFCBDE80840FFF753BC000010B50139EB
:1039F0000244904201D1002010BD10F8013B11F8A3
:103A0000014FA342F5D0181B10BD0000034611F86A
:103A1000012B03F8012B002AF9D170471210121361
:103A20001211000001105A00031059000120580023
:103A30000320560053544D333248373F3F3F005325
:103A4000544D3332483734332F37353300000000BC
:103A5000000000000D110008F910000835110008E1
:103A6000211100082D110008191100080511000886
:103A7000F110000891110008000000000100000092
:103A8000000000006D61696E00000000A43A0008AB
:103A9000682400206026002001000000B51A0008FC
:103AA0000000000069646C65000000000200000076
:103AB0000000000039130008A51300084000400072
:103AC000F82A0020082B002002000000000000005F
:103AD0000300000000000000E913000800000000DF
:103AE00010000000182B0020000000000100000062
:103AF00000000000882D0020010102006D526F00BF
:103B000025424F415244252D424C002553455249F0
:103B1000414C25007D1E0008E51D0008A512000887
:103B2000611E0008430000002C3B0008090243000E
:103B3000020100C032090400000102020100052454
:103B400000100105240100010424020205240600DE
:103B500001070582030800FF09040100020A0000B2
:103B60000007050102400000070581024000000037
:103B700012000000783B0008120110010200004012
:103B80000912415700020102030100000403090465
:103B900025424F41524425006D526F436F6E74723F
:103BA0006F6C5A65726F436C617373696300303177
:103BB00032333435363738394142434445460000C4
:103BC000000000005915000839180008E518000821
:103BD00040004000C02E0020C02E00200100000048
:103BE000D02E0020800000004001000008000000EE
:103BF0000001000000040000080000000000802A0E
:103C000000000000AAAAAAAA00000000FFFF00000E
:103C10000000000000A00A004401000000000000B5
:103C2000AAAAAAAA00000000FFFF000000000000EE
:103C3000000000000000000000000000AAAAAAAADC
:103C400000000000FFFF0000000000000000000076
:103C50000040100000000000AAAA8AAA004010003C
:103C6000FFFF000000000000000000000000004016
:103C700000000000AAAAAAAA00000040FFFF00005E
:103C80000000000000000000010010000000000023
:103C9000AAAAAAAA01001000FFFF0000000000006D
:103CA000000000004000040000000000AAAAAAAA28
:103CB00040000400FFFF00000000000000000000C2
:103CC0000000000000000000AAAAAAAA000000004C
:103CD000FFFF0000000000000000000000000000E6
:103CE00000000000AAAAAAAA00000000FFFF00002E
:103CF00000000000000000000000000000000000C4
:103D0000AAAAAAAA00000000FFFF0000000000000D
:103D1000000000000000000000000000AAAAAAAAFB
:103D200000000000FFFF0000000000000000000095
:103D3000FF00000000000000343A00083F000000CF
:103D4000500400003F3A00083F00000000960000C9
:103D500000000800040000008C3B00080000000088
:103D60000000000000000000000000000000000053
:043D7000000000004F
:00000001FF
